:100000000C94DB010C9413020C9413020C94130255
:100010000C9413020C9413020C9413020C9413020C
:100020000C9413020C9413020C94EB1D0C94BD1E43
:100030000C94DF180C9413020C9413020C9413020A
:100040000C9413020C9413020C9413020C941302DC
:100050000C9413020C9467190C9413020C94130261
:100060000C9413020C9413020C9413020C941302BC
:100070000C9413020C9413020C9413020C941302AC
:100080000C9413020C9413020C9413020C9413029C
:100090000C9413020C9413020C9413020C9413028C
:1000A0000C9413020C9413020C941302DB04DB0473
:1000B000070507056F058D05A506A50698053106F8
:1000C000420642062A1F511F4920511F49209D1FE9
:1000D000C01F492017202620A8001E001F00200056
:1000E00021002200230024002500260027002A00EA
:1000F0005300380055002D00290014001A00080094
:10010000150017001C0018000C00120013004C0012
:100110005F006000610057002B000400160007001C
:1001200009000A000B000D000E000F003300340020
:100130005C005D005E002E0039001D001B00060003
:1001400019000500110010003600370038002800A3
:1001500059005A005B005800E100E000E200E300B3
:100160002C412C002C002C425000510052004F001A
:1001700062006200630058003500000000000000CB
:10018000000000000000000000000000000000006F
:10019000000000000000000001003A003B003C00AD
:1001A0003D003E003F0040004100260227020100C2
:1001B000010001000100005C3500420043004400E2
:1001C0004500010001002D002E002F0230023102F7
:1001D0000100010001000100010001000100010017
:1001E0000100010001000100010001000100010007
:1001F00001000100010001000100010001000100F7
:10020000010001000100010001004A004D00010051
:1002100001000100010001000100010001000100D6
:100220000100010001000100AB00AA00A900AE001E
:1002300001000100010001000100000000000000B9
:1002400000000000000000000000000000000000AE
:1002500000000000000000003C034400690073003F
:1002600061007200720061007900200028004F00D8
:100270007200740068006F006C0069006E00650019
:100280006100720020004C00610079006F00750071
:10029000740029000000120353006E006500610025
:1002A0006B0062006F00780000000403090409027B
:1002B0003B00020100A0FA09040000010301010053
:1002C00009211101000122400007058103080001F6
:1002D00009040100010300000009211101000122AD
:1002E0007B000705820320000112010002000000CC
:1002F000084253030001000102000105010902A1A7
:100300000185020901A10005091901290815002527
:100310000195087501810205010930093115812512
:100320007F95027508810609381581257F9501752D
:10033000088106050C0A38021581257F950175088C
:100340008106C0C005010980A101850319012AB7F2
:1003500000150126B700950175108100C0050C0934
:1003600001A101850419012AA002150126A0029508
:100370000175108100C005010906A101050719E0FA
:1003800029E7150025019508750181029501750879
:1003900081010507190029FF150026FF0095067544
:1003A0000881000508190129059505750191029537
:1003B0000175039101C011241FBECFEFDAE0DEBF4B
:1003C000CDBF04B603FE18C08091A6029091A7028B
:1003D000A091A802B091A9028730904BA740B04BE2
:1003E00059F41092A6021092A7021092A80210923D
:1003F000A902E0E0F8E3099511E0A0E0B1E0E8EF40
:10040000F1E402C005900D92A23AB107D9F722E0BB
:10041000A2EAB1E001C01D92A63AB207E1F70E943C
:10042000C9120C94FA200C940000823038F4662330
:1004300011F08AEA01C089EA0E94890481E00895E6
:1004400081E0089581E008950C94220208950C94AF
:1004500026021F93CF93DF9300D000D01F92CDB719
:10046000DEB749835A836B833091A50189819A81D4
:10047000311114C0662359F0222349F00E94E2088A
:10048000182F682F89819A810E948B0803C00E94CF
:10049000B608182F69817A81812F04C00E94E20872
:1004A00069817A810F900F900F900F900F90DF91DC
:1004B000CF911F910C943210FC01262F4081518165
:1004C0006281738184810C94290281E00895CF9325
:1004D000DF93EC0160E00E945C02BE01DF91CF91EE
:1004E0000C9427020C947A110C94761108950E94B2
:1004F00035070E9476022FEF84E39CE02150804074
:100500009040E1F700C000000C948D190F931F93E9
:10051000CF93DF938C0161E00E945C02EC01B80193
:100520000E9424028823F1F1B801CE010E94AA178B
:100530008823C1F1B801CE010E945F15882391F193
:10054000B801CE010E940617882361F1F80182816B
:10055000882309F1CB358DE5D807C1F050F4C115DA
:10056000FCE5DF0781F0CF3DDC45A9F40E94190EC0
:1005700019C0CC35EDE5DE0761F0CD35DD4559F428
:100580000E945C0D08C00E9477020CC00E94650D9D
:1005900002C00E94680DC801DF91CF911F910F9199
:1005A0000C94200280E0DF91CF911F910F9108956C
:1005B0000E94C1180C94FE020E9401030C94C718FB
:1005C00008950C94E00281E00895CF93C82F0E9413
:1005D000E302882329F0C0FF02C0299A01C02998AC
:1005E000CF910895219A29980895CF93C82F0E94FA
:1005F000E1028C2F0E94E502CF91089580E00C94D7
:10060000F5020E9406180C94F5020E9406189091BB
:10061000A401891721F08093A4010C94F502089598
:10062000CF93DF93CDB7DEB72B970FB6F894DEBF2D
:100630000FBECDBF4F83588769877A878B8761113B
:100640000E94A80C9E012F5F3F4F86E0F901119296
:100650008A95E9F785E0FE013796D90101900D9260
:100660008A95E1F789819A814C815D81452B31F032
:100670009F3F31F491E08F3F19F403C091E001C036
:1006800090E090FF09C049815A816B817C818D8106
:100690009E810E94C90B05C0C9010E94650281119B
:1006A000F2CF2B960FB6F894DEBF0FBECDBFDF9111
:1006B000CF910895FC01808191810E9424090895C1
:1006C000CF93882309F4A4C0C82F8238C1F40E94B4
:1006D000061881FD9DC069E380910201909103019C
:1006E0000E9499180E94CA0C2FEF81EE94E02150CD
:1006F00080409040E1F700C0000069E319C08338F2
:1007000001F50E94061880FD83C063E58091020117
:10071000909103010E9499180E94CA0C2FEF81EE5C
:1007200094E0215080409040E1F700C0000063E574
:1007300080910201909103010E949B18CF910C942B
:10074000CA0C8438C1F40E94061882FD61C067E4B7
:1007500080910201909103010E9499180E94CA0C95
:100760002FEF81EE94E0215080409040E1F700C0EF
:10077000000067E4DDCF8CEF8C0F813AD0F46C2F52
:1007800080910201909103010E946318882349F02F
:100790006C2F80910201909103010E949B180E948E
:1007A000CA0C6C2F80910201909103010E9499184C
:1007B000C5CF80E28C0F883048F4C77081E001C05B
:1007C000880FCA95EAF70E948B0CB8CFEBE5EC0FC7
:1007D000E33040F4F0E0E95BFE4F808190E0CF91A0
:1007E0000C942B18E8E5EC0FE73150F4F0E0EE0F35
:1007F000FF1FE75EFE4F80819181CF910C944118DD
:10080000CD3E30F08C2F0E944E13CF910C942014CB
:10081000CF910895882309F464C0823879F40E9446
:10082000061881FF5EC069E3809102019091030187
:100830000E9499180E94CA0C69E310C08338B1F471
:100840000E94061880FF4DC063E5809102019091DF
:1008500003010E9499180E94CA0C63E5809102016D
:10086000909103010E949B180C94CA0C843879F46F
:100870000E94061882FF35C067E4809102019091C2
:1008800003010E9499180E94CA0C67E4E7CF9CEF0D
:10089000980F913A10F4682FE1CF90E2980F9830BA
:1008A00050F4877091E001C0990F8A95EAF7892F7B
:1008B0000E94910CD9CF9BE5980F933020F480E0F3
:1008C00090E00C942B1898E5980F973120F480E075
:1008D00090E00C9441188D3E20F00E94A9130C94D6
:1008E000201408951F93CF93DF93182FEB010E94DC
:1008F0006003209741F08FE99FE00197F1F700C076
:1009000000002197F6CF812FDF91CF911F910C949A
:100910000A04893319F060E070E002C060E570E01D
:100920000C947204882321F00E948B0C0C94CA0C46
:100930000895882321F00E94910C0C94CA0C08950C
:10094000CF92DF92EF92FF920F931F93CF93DF939B
:100950007C01D62FC72FFC011281058102950F70F3
:100960000E94810C8823B9F01123A9F08C2F807F7D
:10097000803421F080E28D0F883068F080917C0215
:1009800082FD09C082E00E942A0D0E94810C91E044
:10099000D82ED92601C0D12CCC2EC2948FE0C822EB
:1009A0008C2D90E08C30910508F0CFC1FC01EA5A03
:1009B000FF4F0C9491208C2F807FCF70882311F0F3
:1009C000C295C07F112399F0CC2309F4AAC180E21B
:1009D0008D0F883010F0D11104C08C2F0E948B0C29
:1009E00003C08C2F0E949B0C0E94CA0C9AC18D2FB1
:1009F0000E940A04CC2309F4A8C180E28D0F88303C
:100A000038F1DD2329F18C2F0E94A10C24C08C2FFA
:100A1000807FCF70803211F0C295C07FDD2319F046
:100A2000D130A1F13DC080917C0282FF17C011231B
:100A300049F0CC2329F08C2F0E948B0C0E94CA0C09
:100A400080E070C180E00E940A04CC2309F47DC1DB
:100A50008C2F0E94910C0E94CA0C77C1112371F057
:100A6000002341F0013031F40E94AB0C8C2B0E942A
:100A7000B30C6BC10E94AB0C8C2B1DC0002319F072
:100A8000013009F462C10E94C00C25C0112321F07D
:100A9000063008F05AC10EC0053008F056C11BC020
:100AA000112361F0002331F0F701858180FF39C106
:100AB0008F7085838C2F0E94920447C1002359F0C8
:100AC000D93309F03FC1FFEF07EE13E0F1500040CA
:100AD0001040E1F735C18C2F0E94990436C18C2F4C
:100AE00086958695837019F0813061F02EC11123AF
:100AF00021F08D2F9C2F937002C080E090E00E9427
:100B00002B182BC1112321F08D2F9C2F937002C025
:100B100080E090E00E94411820C18D2F112319F030
:100B20000E944E1302C00E94A9130E94201415C1F6
:100B30008C2F837009F047C011110BC12D2F229506
:100B400026952770220F220F6D2F6F70862F90E051
:100B5000A0E0B0E0022E04C0880F991FAA1FBB1F9F
:100B60000A94D2F7D4FF10C04FE050E060E070E08C
:100B700004C0440F551F661F771F2A95D2F7409572
:100B800050956095709503C040E050E0BA01C6955D
:100B9000C695C3708A019B01082B192B2A2B3B2B6E
:100BA000C901B801C23049F058F4C13019F00E94AF
:100BB000A107CFC00E948F07CCC00E94B307C9C055
:100BC0000E948D07C6C0112319F08C2F817001C0BF
:100BD0008695882309F4BDC02D2F22952695277070
:100BE000220F220F6D2F6F70862F90E0A0E0B0E0F3
:100BF000022E04C0880F991FAA1FBB1F0A94D2F7A8
:100C0000D4FF10C04FE050E060E070E004C0440F3B
:100C1000551F661F771F2A95D2F74095509560950E
:100C2000709503C040E050E0BA01C695C695C37008
:100C30008A019B01082B192B2A2B3B2BC901B801D8
:100C4000C23049F058F4C13019F00E94660881C0E2
:100C50000E9454087EC00E9478087BC00E94C7078B
:100C600078C0CF70112339F08C2F0E94ED078D2FA3
:100C70000E9492046EC08D2F0E9499048C2F0E94B6
:100C80000E0867C0D23F21F128F4D03F41F0D13F98
:100C9000C1F043C0D33F19F1D43F79F03EC01123D6
:100CA00041F0053008F051C08C2F8F710E9433083D
:100CB0004CC0063008F049C0F7CF80917C0282FF1B
:100CC00018C0112339F08C2F8F710E94ED073DC0A1
:100CD0001123C9F38C2F8F710E940E0836C0112387
:100CE00029F08C2F8F710E94D8072FC00E94D30744
:100CF0002CC0112349F0CF718C2F0E94ED0763E0C7
:100D00008C2F0E940F0D21C081E00E942A0D02301D
:100D1000E0F082E00E942A0D18C0112331F0002378
:100D200091F28D2F0E94600310C0002399F2D933F5
:100D300049F41FEF27EE33E0115020403040E1F737
:100D400000C000008D2F0E940A0488EF8C0D8430B3
:100D500020F40E9406180E94F502DD20C9F00E94CE
:100D60007D0C80FD15C0F70112820E94770C0E9455
:100D7000ED07C7010E94E9060E94770CDF91CF9131
:100D80001F910F91FF90EF90DF90CF900C940E0881
:100D9000DF91CF911F910F91FF90EF90DF90CF9057
:100DA00008950F931F93CF93DF93EC0168817981AE
:100DB0008A810E942F098C010E948A080E947B0769
:100DC000B801CE010E94A004DF91CF911F910F9135
:100DD0000895CF93DF93EC01988189812B813C8129
:100DE000232B31F08F3F31F481E09F3F19F403C092
:100DF00081E001C080E080FD1DC0CE010E9486021E
:100E0000811110C00E94810C8823A1F08A8188235F
:100E100089F080917C0282FD0DC082E0DF91CF914C
:100E20000C942A0DCE010E94D106CE01DF91CF9104
:100E30000C946702DF91CF91089580E090E00E94CA
:100E40002B1880E090E00E9441180E94A80C0E949C
:100E5000CA0C0E9451150C942014809102019091AB
:100E600003010E949D180C941D070E94980C0C947D
:100E70002D0792959F70963079F010F4925001C032
:100E80009A50923068F4803F69F018F4883E40F43C
:100E900009C0843F29F406C0883E20F0813F11F04C
:100EA00080E0089581E00895FC01808191810E9495
:100EB00024090E9439070895CF93DF9300D000D012
:100EC0001F92CDB7DEB70F900F900F900F900F903D
:100ED000DF91CF910895CF93DF9300D000D000D061
:100EE000CDB7DEB726960FB6F894DEBF0FBECDBFE6
:100EF000DF91CF910895089508950C947C070C9488
:100F00007D070E947F076093E6017093E70180935D
:100F1000E8019093E9010C941D070C9481070F934D
:100F20001F930091E6011091E7012091E8013091B3
:100F3000E901602B712B822B932B1F910F910C9445
:100F400081070F931F930091E6011091E701209113
:100F5000E8013091E90160237123822393231F91DB
:100F60000F910C9481070F931F930091E60110914C
:100F7000E7012091E8013091E9016027712782277C
:100F800093271F910F910C9481070C947C070E946A
:100F9000C5076093E2017093E3018093E4019093AD
:100FA000E5010C941D0760E070E0CB010C94C707CD
:100FB0000F931F9341E050E060E070E08A019B01D5
:100FC00004C0000F111F221F331F8A95D2F7C901D9
:100FD000B8011F910F910C94C7070F931F9341E025
:100FE00050E060E070E004C0440F551F661F771F9B
:100FF0008A95D2F78091E2019091E301A091E401FA
:10100000B091E5018A019B01082B192B2A2B3B2B60
:10101000C901B8011F910F910C94C7070F931F933B
:1010200041E050E060E070E004C0440F551F661FCF
:10103000771F8A95D2F7409550956095709580916D
:10104000E2019091E301A091E401B091E5018A01F0
:101050009B01082319232A233B23C901B8011F91AF
:101060000F910C94C7070F931F9341E050E060E08D
:1010700070E004C0440F551F661F771F8A95D2F792
:101080008091E2019091E301A091E401B091E5012A
:101090008A019B01082719272A273B27C901B80184
:1010A0001F910F910C94C7070F931F930091E201BA
:1010B0001091E3012091E4013091E501602B712B47
:1010C000822B932B1F910F910C94C7070F931F93A3
:1010D0000091E2011091E3012091E4013091E501DA
:1010E00060237123822393231F910F910C94C707D0
:1010F0000F931F930091E2011091E3012091E4010D
:101100003091E50160277127822793271F910F9166
:101110000C94C707089520E1929F800D1124E82FB9
:10112000E695E695E695877051E001C0550F8A95E2
:10113000EAF785E0E89FF0011124EA55FE4F20E030
:1011400030E070E04081CB01022E02C09695879579
:101150000A94E2F7817081958427852384278193FF
:101160002F5F3F4F2530310569F7089520E1929FA9
:10117000800D1124682F669566956695982F977057
:1011800085E0689FB001112440E050E080E0FB0161
:10119000E40FF51FEA55FE4F208130E0092E02C012
:1011A000369527950A94E2F721703327042E01C063
:1011B000220F0A94EAF7822B4F5F5F4F45305105AB
:1011C00031F70895BF92CF92DF92EF92FF920F9383
:1011D0001F93CF93DF938C01C090E201D090E30185
:1011E000E090E401F090E5018091E6019091E70143
:1011F000A091E801B091E901C82AD92AEA2AFB2A7C
:10120000CFE1D0E0D701C6010C2E04C0B695A7955A
:10121000979587950A94D2F780FD04C0219790F79F
:10122000B12C07C0BC2EB8018C2F0E94471001972B
:10123000A9F38B2DDF91CF911F910F91FF90EF902C
:10124000DF90CF90BF900895CF93DF93EC010E9481
:10125000E208BE010E944710DF91CF9108951F93CD
:10126000CF93DF93EB019091A501992321F0CB015E
:101270000E94240913C0882349F0CB010E94E20890
:10128000182F682FCE010E948B0804C0CB010E944A
:10129000B608182FBE01812F0E944710DF91CF9111
:1012A0001F9108951F93CF93DF93C091EA0116E039
:1012B0008091EB01C81799F0D0E01C9FF0011D9FB1
:1012C000F00D1124E451FE4F408151816281738100
:1012D000848195810E946B072196C770E9CFDF91C9
:1012E000CF911F91089540911C0250911D02609171
:1012F0001E0270911F0280912002909121020C9495
:101300006B07EF92FF920F931F93CF93DF93809120
:10131000210282958F7009F065C080911E0288239A
:1013200009F460C08091EA01F090EB0110911C0279
:1013300000911D0260911F027091200291E01F3FF9
:1013400009F090E0C0910001D0910101292F96E0B1
:10135000E92E8F1509F446C06115710521F00F3F84
:1013600021F030E003C031E001C0322F90E030FDC9
:1013700036C0E89EF001E99EF00D1124DF01A45172
:10138000BE4F11963C911197301329C03C913113F7
:1013900026C012963C911297311121C013964D919F
:1013A0005C911497461B570B4C175D07C0F4809156
:1013B00021028F70806180932102EF50FE4F808167
:1013C0008F70806180838CE192E00E94E906DF915A
:1013D000CF911F910F91FF90EF900C9452090196BD
:1013E0008770B7CFDF91CF911F910F91FF90EF9052
:1013F00008959F92AF92BF92CF92DF92EF92FF92A9
:101400000F931F93CF93DF93CDB7DEB761970FB6DE
:10141000F894DEBF0FBECDBF8C0185E0F801DE0180
:101420001D9601900D928A95E1F7D8011296EC90E5
:1014300090911C02E0911D0220911F023091200228
:101440002115310531F0EF3F31F481E09F3F19F470
:1014500003C081E001C080E0B82FB1709B2E80FDF9
:1014600047C1D8014C9111965C9111971396AD909C
:10147000BC9014978CE1C82E82E0D82EF0901E020A
:10148000B501621B730B2091000130910101FF2017
:1014900009F4D9C0809121026217730708F095C042
:1014A000282F207F09F052C05E1313C0491311C0CA
:1014B000FE2CE1100EC08F708061809321020E948B
:1014C0007309C6010E94E90680912102F801858313
:1014D0004DC1AB2831F05F3F31F481E04F3F19F44B
:1014E00003C081E001C080E080FD03C081E08E2563
:1014F00002C080E090E0F82FF170FF2E80FF1CC04A
:101500008091EA012091EB0136E0821709F40BC1CA
:1015100090E0389FF001399FF00D1124E451FE4F07
:101520006181561306C06081461303C06281E612D2
:1015300003C001968770E9CFFE2CEE2009F416C196
:101540008091210281608093210254C05E1306C005
:10155000491304C0E11002C0F80199C0C8010E94FB
:101560005407882361F1EE2051F120912102822F4E
:1015700082958F7090E0029774F080911C02909198
:101580001D0298878F831986BB86AA862C87CE0179
:1015900007960E94E90686E0F801ACE1B2E001900E
:1015A0000D928A95E1F70E9481090E9473090AC091
:1015B0005E1711F1C8010E94540781112CC0C801A7
:1015C0000E94E906FF24F394D1C0282F207F81F7E1
:1015D0007A2DB98AA88A6E2D89890E945C078CE1D0
:1015E00092E00E94E90686E0D6011D928A95E9F70D
:1015F0000E947309F12CBAC04913DCCFE110DACF95
:10160000F8018583C8010E94E90686E0D6011D9293
:101610008A95E9F7ABC0EE2091F220912102822F4A
:1016200082958F7090E002970CF4B5CF80911C02E8
:1016300090911D029A8389831B82BD82AC822E8386
:10164000CE010196A6CF6217730708F044C0FE2CA6
:10165000EE2009F4B4CF5E1330C049132EC02091A0
:10166000210220FD21C0822F82958F70482F50E0EB
:1016700041155105C9F0F80125834F30510541F05E
:101680008F5F982F9295907F822F8F70892B858303
:10169000C8010E94E90686E0F801ACE1B2E00190E1
:1016A0000D928A95E1F73CC086E0F801ACE1B2E02A
:1016B00001900D928A95E1F759C0C8010E94540724
:1016C000811169CF80912102816080932102C8013C
:1016D0000E94E9064BC07A2DB98AA88A6E2D8989A5
:1016E0000E945C0786E0D6011D928A95E9F718C032
:1016F000EE2009F464CFC8010E945407F82E882315
:1017000009F45DCF86E0F801ACE1B2E001900D9202
:101710008A95E1F78CE192E00E945A030E948109C8
:101720000E94730923C04D875E878D859E850E9428
:101730002409292F22952F70223028F49F7039F028
:10174000811105C00BC0243028F49F7049F4805EDD
:10175000883020F0C8010E94E9069F2CF92C06C0B1
:10176000D80115969C91907F91F7F8CF8F2D6196B7
:101770000FB6F894DEBF0FBECDBFDF91CF911F91A2
:101780000F91FF90EF90DF90CF90BF90AF909F9020
:1017900008951F93CF93DF93CDB7DEB72C970FB685
:1017A000F894DEBF0FBECDBF4F83588769877A8715
:1017B0008B879C87CE0107960E94F9098823D1F078
:1017C0009F8188852A853B85232B31F08F3F31F41B
:1017D00081E09F3F19F403C081E001C080E080FDFB
:1017E00047C04F81588569857A858B859C850E9485
:1017F0006B073EC086E0FE013796DE011196019030
:101800000D928A95E1F7FF81E8856A857B856115F0
:10181000710531F0EF3F31F481E0FF3F19F403C06F
:1018200081E001C080E080FD23C02091EB0130E029
:10183000C9010196877099274091EA0150E0841709
:101840009507F1F1F983EA837D836C8396E0929F9B
:10185000D001939FB00D1124A451BE4FFE013196CB
:1018600001900D929A95E1F78093EB010E94520945
:1018700016E08091EA019091EB01891771F1189FB0
:10188000C001112484519E4F0E94F909882329F137
:10189000E091EA011E9FF0011124E451FE4F4081C6
:1018A000518162817381848195810E946B0780914F
:1018B000EA0190E00196877099278093EA01D9CFD9
:1018C0000E9435071092EB011092EA01ECE1F2E080
:1018D00086E0DF011D928A95E9F72C960FB6F89401
:1018E000DEBF0FBECDBFDF91CF911F9108958091D4
:1018F0002A02859585958595089580912A0287709D
:10190000089590912A02977081E009F480E008958B
:1019100080913502089590913502892B809335028C
:10192000089580959091350289238093350208951A
:1019300010923502089590913402892B80933402DD
:1019400008958095909134028923809334020895FC
:1019500010923402089580912B02089508950C94FA
:10196000AE0C0C94AF0C90917C0292FD08C090914B
:101970002B02981721F080932B020C94B10C089540
:1019800080912B02882329F010922B0280E00C9486
:10199000B10C0895CF93DF93E0910201F091030120
:1019A000809135028083E0910201F09103019081E2
:1019B00080913402892B808380912B02882381F0CF
:1019C000E0910201F09103019081892B8083809145
:1019D0000201909103010E94571881110E94C00CCE
:1019E000C0910201D091030148E050E062E272E050
:1019F000CE010E94AB20892B69F088E0FE01A2E2B3
:101A0000B2E001900D928A95E1F7CE01DF91CF917E
:101A10000C941218DF91CF9108950C94AE0C909114
:101A20007C0292FD10C098E0899F90011124262B22
:101A300020932A020E94ED0780912A0285958595C0
:101A400085950C940D0D0C94ED0710922A0280E000
:101A50000C940D0D20912A028095822380932A02F6
:101A6000982F977099F430E0482F082E000C550BF2
:101A70002417350759F090917C0292FD07C0859597
:101A8000859585950E940E080C94250D08959091DA
:101A90007C0292FB222720F9281769F080FB92F93B
:101AA00090937C0280917B0290917C020E94950D24
:101AB00082E00C942A0D089580917C0282FB882795
:101AC00080F991E089270C94470D81E00C94470D33
:101AD00080E00C94470D6FEF7FEF80E090E00C9476
:101AE000E42080E090E00E94C02021E0893E9E4FEB
:101AF00009F020E0822F089582E090E00C94B82055
:101B000083E090E00C94B820CF9384E090E00E94B2
:101B1000B820C82F82E290E00E94B8202C2F30E03D
:101B2000A901582BCA01CF910895CF93C92F682FCF
:101B300084E090E00E94C6206C2F82E290E0CF917A
:101B40000C94C620AB01BC018FE090E00C94D8202F
:101B5000AB01BC0183E190E00C94D82060E070E020
:101B6000CB010C94A80D60E070E0CB010E94A20DA7
:101B70000C94AE0D69EE7EEF80E090E00E94E420D0
:101B800060E082E090E00E94C62060E083E090E0A8
:101B90000E94C6201092E6011092E7011092E8011F
:101BA0001092E90160E084E090E00E94C62060E0CD
:101BB00082E290E00E94C62060E085E090E00E9412
:101BC000C62060E086E090E00E94C6206FEF87E0CC
:101BD00090E00E94C62040E050E0BA0188E090E02A
:101BE0000E94D82060E08DE090E00E94C62040E096
:101BF00050E0BA0188E190E00E94D82060E087E1DF
:101C000090E00E94C62040E050E0BA018CE190E0F4
:101C10000E94D82060E070E080E290E00E94E42022
:101C200040E050E0BA0188E190E00E94D8200C9496
:101C3000B30D0C94BA0D682F8EE090E00C94C62082
:101C40000E944C1960934A0270934B0280934C029D
:101C500090934D026093460270934702809348022E
:101C60009093490208950E944C1960934A02709320
:101C70004B0280934C0290934D026093420270930A
:101C800043028093440290934502089585B780688B
:101C900085BF85B7806885BF089581E008950C945D
:101CA0004D0E08950C94510E0C94510E0C94540E3C
:101CB0000C94510E0C94580E0C94510E0E94460E2A
:101CC00083E291E10E94FC170E945C0E0C945A0E74
:101CD0000E94520E0C94510E0E943D110C94F2027F
:101CE0000E9437190E9422120E946C0E0E94B016A8
:101CF0000C94560E5F926F927F928F929F92AF924A
:101D0000BF92CF92DF92EF92FF920F931F93CF93E8
:101D1000DF93CDB7DEB72A970FB6F894DEBF0FBEBC
:101D2000CDBF0E943712C82E81110E94200E36E3CB
:101D3000832E32E0932E00E010E0502E802F0E9480
:101D400061115C01F401619071904F016826792660
:101D500061147104B1F40F5F1F4F0630110569F76C
:101D60008FEF89838A831B820E9440198160782FBC
:101D70009D838C8349815A816B818D810E941003E0
:101D80003AC080914E0281FD0E946A11D12CEE244E
:101D9000E394F12CC3018E219F21892B29F10E940C
:101DA0004F0E8823A9F0DE825F82AE20BF2081E043
:101DB000AB2809F480E088870E9440198160782F61
:101DC0009A8789874E815F8168858A850E94100382
:101DD000000F111FF801EA5CFD4F80819181E82618
:101DE000F926F182E08207C0D394EE0CFF1CF0E1EB
:101DF000DF12D0CFB0CF81E0C11001C080E02A96C1
:101E00000FB6F894DEBF0FBECDBFDF91CF911F910B
:101E10000F91FF90EF90DF90CF90BF90AF909F9089
:101E20008F907F906F905F9008950E947A0E0E942D
:101E3000C31681110E94330E0E943E140C940503B8
:101E4000CF93DF930E944C10EC01811521E592079E
:101E500008F045C0811530E5930708F094C0883E2E
:101E6000910528F5803E910508F0F8C0883A910563
:101E700070F4853A910508F07CC08130910509F431
:101E800075C008F4E8C0049708F0E8C0E4C08F3BD0
:101E9000910508F0E0C0C85AD0E0CC0FDD1FC65B4A
:101EA000DE4F0990D881C02DCE019464D8C0811531
:101EB00040E2940758F4811551E0950708F0CEC030
:101EC0008D3E910508F4C7C09065C9C0C11580E476
:101ED000D80708F4C0C0DF70CE01906AC0C0811579
:101EE00025E59207A8F4811534E5930708F095C01D
:101EF000811543E5940708F07BC0811552E59507ED
:101F000008F061C0D82FCC27CE01816F906AA7C09E
:101F1000C11589E5D807A0F4C11528E5D20708F056
:101F200082C0C11536E5D30708F095C08C2F0E94FA
:101F3000E0108F7190E0D82FCC27CE0190628FC037
:101F4000C1154AE5D40708F474C0CE019056811536
:101F5000904208F080C08D2F8F710E94E010DD2725
:101F6000D0628F71AE01582BCA0179C081E090E038
:101F700076C0C55AD0E0C858DE4F8881C82FD0E05F
:101F8000CE0190646CC074E0969587957A95E1F7E0
:101F9000282F23703C2F337081E090E002C0880F1F
:101FA000991F3A95E2F79C68AC01522B9A019C2F3D
:101FB0009F709695969550E2959FE0011124C90176
:101FC0008C2B9D2B4CC08370992721E030E002C000
:101FD000220F331F8A95E2F79C2F9695969580E203
:101FE000989FE0011124C22BD32BCE019C6837C0EF
:101FF0008370992721E030E002C0220F331F8A95B9
:10200000E2F79C2F9695969540E2949FE00111246B
:10201000C22BD32BCE019A6822C0D82FCC27CE0159
:10202000846F906A1CC0DC2FCC27CE01806F906A31
:1020300016C08C2F8F700E94E01094E0D695C79543
:102040009A95E1F7CF70D0E0DC2FCC27D0699E01C4
:10205000282BC90104C080E090E001C0CE01DF91CF
:10206000CF910895E72FF0E096E0899FE00DF11DF4
:10207000112484E0EE0FFF1F8A95E1F7E60FF11DB2
:10208000EE0FFF1FE852FF4F8591949108950E9433
:1020900032100E94200F08958238910569F1B0F442
:1020A0008133910509F46DC048F48932910509F432
:1020B00063C08A32910509F469C00895853391059A
:1020C00009F455C089339105B9F00895833E91050F
:1020D00069F138F4803E9105B1F0823E910509F135
:1020E0000895863E9105A9F1873E9105B9F1843E98
:1020F000910509F064C023C020917B0220FD4FC0F0
:1021000021FD4DC0089580917B0280FD44C08091E7
:102110007C0280FF44C080917B0284FD42C083EE3C
:102120004DC080917B0282FF38C0F5CF80917B0249
:1021300082FD33C080917C0280FD31C0ECCF809164
:102140007C0281FF32C080917B0284FD2AC087EE31
:1021500035C080917B0283FF26C0F5CF80917B0242
:1021600083FD21C080917C0281FD1FC0ECCF809156
:102170007B0285FD1CC01DC080917B0285FD19C0BE
:1021800016C080917B0286FD16C017C080917B022D
:1021900086FD13C010C089E311C082EE0FC080EE2F
:1021A0000DC080E00BC086EE09C084EE07C089E256
:1021B00005C085E303C08AE201C081E390E0089591
:1021C00090917B0292FF0DC0282F2871283019F4BE
:1021D000877F846006C0282F2471243011F48B7F00
:1021E000886093FF0DC0282F2871283119F4877E4D
:1021F000846106C0282F2471243111F48B7E8861FC
:1022000020917C0220FF0DC0382F3871383019F42E
:10221000877F816006C0382F3171313011F48E7F95
:10222000886021FF0DC0282F2871283119F4877E7E
:10223000816106C0282F2171213111F48E7E8861C1
:1022400094FD877E089580E008950C946B0D0E94A4
:1022500037128FE39CE90197F1F700C000000E945C
:10226000371281E00E94611180FF04C00E94251195
:102270000C948D1908950C9427110E94710D8111F1
:1022800002C00E94190E0E947C0D80934E020E9493
:10229000840D90937C0280937B020E943B110E94EC
:1022A000800D682F70E080E090E00E948D076091C3
:1022B000E2017091E3018091E4019091E5010C94B9
:1022C000C507E82FF0E0EE0FFF1FE757FD4F8081B5
:1022D00091810895089580EA8A95F1F7089500C0E4
:1022E00008950C946B1108950C9473110C9474114F
:1022F0000C9473110C947811F894E82FE295EF7018
:10230000F0E031A1282F2F7081E090E001C0880F0C
:102310002A95EAF7982F9095932391A392A1892B60
:1023200082A3789408950F931F93CF93DF93CBE804
:10233000D1E089918F3F11F00E947C1181E0C13979
:10234000D807B9F7CBE7D1E00BE811E089918F3FCF
:1023500011F00E947C110C171D07C1F7DF91CF917E
:102360001F910F910895BF92CF92DF92EF92FF924B
:102370000F931F93CF93DF938C01C62FD0E0CE0134
:1023800085579E4F6C01FC0190819F3F09F450C01E
:10239000B62EF894E92FE295EF70F0E081A19F70DE
:1023A00021E030E001C0220F9A95EAF7822B81A349
:1023B00082A12095282322A378940E946F11EBE735
:1023C000F1E04BE851E021E030E0E12CF12C6191AB
:1023D0006F3F89F0A62FA295AF70B0E090968C91D8
:1023E00090E06F7002C0959587956A95E2F780FD41
:1023F00002C0C90102C080E090E0E82AF92A220F59
:10240000331F4E175F0719F7F60180818F3F11F0D8
:102410000E947C1161E0E114F10409F460E08B2D6D
:102420000E947111CC0FDD1FC00FD11FF982E8820D
:10243000DF91CF911F910F91FF90EF90DF90CF90A0
:10244000BF9008950E9493118CE0E9E8F2E0DF016B
:10245000982F1D929A95E9F7EDE7F2E0DF011D92C2
:102460008A95E9F786E00E9482120C947202FF922C
:102470000F931F93CF93DF93CDB7DEB72C970FB693
:10248000F894DEBF0FBECDBF8E010F5F1F4F8CE0F3
:10249000F80111928A95E9F7F12C6F2DC8010E947D
:1024A000B311F394F6E0FF12F8CF4CE050E0B8011E
:1024B0008DE792E00E94AB20FF24F394009709F48B
:1024C000F12C892B41F08CE0F801ADE7B2E00190EE
:1024D0000D928A95E1F72F2D46E069E872E08DE7CD
:1024E00092E00E9483120E9474028F2D2C960FB6E8
:1024F000F894DEBF0FBECDBFDF91CF911F910F913A
:10250000FF9008950895FF920F931F93CF93DF9349
:10251000F82E092F162FD72FC42F222349F081E040
:10252000809351020E9440199093500280934F0271
:10253000809151028823D9F080914F0290915002EE
:102540000E945819059798F0EF2DF02FA12FBD2F5D
:1025500080E090E04C2F50E08417950734F42191EF
:1025600031912D933D930196F7CF10925102DF9157
:10257000CF911F910F91FF9008950E94431B0E94DD
:10258000700E0C944F1B0E94531B0E94150F0C944D
:102590006D1B0E94DE180E942A1B0E945E0E0E9484
:1025A000BD120E94C3120E94680EFBCF8091580298
:1025B00080FF06C06091090170E0660F771F26C09A
:1025C00081FF04C06091090184E005C082FF07C05B
:1025D0006091090188E0689FB001112417C09091B3
:1025E00057029923D1F060910801961788F720913E
:1025F000090188E0289F90011124929FA001939FD8
:10260000500D112470E0CA010E947D2060387105D0
:1026100040F46115710519F406C068E070E0862F7A
:1026200008958FE7089581E008958091580280FF12
:1026300008C06091050170E075956795759567957F
:1026400021C081FF06C06091050170E07595679516
:1026500019C082FF04C06091050170E010C0909124
:102660005602992399F0609104019617A0F7809182
:102670000501899FC001112470E00E947D2060380F
:10268000710540F46115710519F406C061E070E050
:10269000862F08958FE7089581E008958D3E21F4F7
:1026A0000E94D612819504C08E3E29F40E94D61253
:1026B00080935C0208958F3E21F40E94D61281958A
:1026C00004C0803F29F40E94D61280935B020895D3
:1026D000893F19F40E94151305C08A3F31F40E9406
:1026E0001513819580935D0208958B3F21F40E941C
:1026F0001513819504C08C3F29F40E941513809313
:102700005E0208959FE0980F983078F421E030E061
:10271000A90102C0440F551F9A95E2F7CA01909192
:102720005A02892B80935A0208958D3F21F480919B
:10273000580281600BC08E3F21F480915802826064
:1027400005C08F3F29F4809158028460809358021D
:1027500008958D3E39F490915C0297FF35C0109238
:102760005C0259C08E3E29F490915C021916BCF3AC
:102770002BC090915B028F3E29F497FF25C01092E9
:102780005B0249C0803F19F41916CCF31DC090912B
:102790005D02893F29F41916BCF410925D023BC01A
:1027A0008A3F19F497FF10C0F8CF8B3F39F490910E
:1027B0005E0297FF09C010925E022DC08C3F21F48B
:1027C00090915E021916BCF39FE0980F983080F448
:1027D00021E030E0A90102C0440F551F9A95E2F7AD
:1027E000CA01809590915A02892380935A0213C09E
:1027F0008D3F21F4809158028E7F0BC08E3F21F4D3
:10280000809158028D7F05C08F3F29F48091580236
:102810008B7F8093580280915B02811106C080916A
:102820005C02811102C01092570280915D028111F9
:1028300006C080915E02811102C010925602089576
:102840000E94401920915B02211104C020915C027A
:10285000222321F0909355028093540220915D022F
:10286000211104C020915E02222321F09093530293
:102870008093520289E592E00C941D18EF92FF922A
:102880000F931F93CF93DF9300D000D000D0CDB72C
:10289000DEB786E0E9E5F2E0DE01119601900D92E7
:1028A0008A95E1F7E0905B02F0905C0200915D0296
:1028B00010915E0210925B0210925C0210925D0217
:1028C00010925E02E11003C0FF2009F45DC0809108
:1028D0005402909155020E945819AC0190915702F0
:1028E000992339F020910A0130E02417350758F078
:1028F0004BC020910B018AE0289F900111242417DE
:10290000350718F041C09F3F19F09F5F9093570221
:10291000EE2061F00E94D6121E1414F09FEF01C049
:1029200091E0989F902D112490935B02FF2061F01D
:102930000E94D6121F1414F09FEF01C091E0989FDF
:10294000902D112490935C0230915B023323E1F0CF
:1029500020915C022223C1F045EB3403C001112415
:10296000992319F090935B0203C081E080935B028E
:1029700035EB2303C0011124992319F090935C02D5
:1029800003C081E080935C02011103C0112309F4AC
:102990005DC080915202909153020E945819AC017F
:1029A00090915602992339F02091060130E02417C6
:1029B000350758F04BC0209107018AE0289F90010D
:1029C00011242417350718F041C09F3F19F09F5F6D
:1029D00090935602002361F00E941513101614F014
:1029E0009FEF01C091E0989F902D112490935D027C
:1029F000112361F00E941513111614F09FEF01C00E
:102A000091E0989F902D112490935E0230915D0289
:102A10003323E1F020915E022223C1F045EB340321
:102A2000C0011124992319F090935D0203C081E045
:102A300080935D0235EB2303C0011124992319F023
:102A400090935E0203C081E080935E0280915B02FE
:102A500081110BC080915C02811107C080915D02E1
:102A6000811103C080915E0281110E942014EB82CB
:102A7000FC820D831E8386E0FE013196A9E5B2E05B
:102A800001900D928A95E1F726960FB6F894DEBF75
:102A90000FBECDBFDF91CF911F910F91FF90EF90AF
:102AA0000895E9E5F2E086E0DF011D928A95E9F7F5
:102AB0001092570210925602109258020895CF9326
:102AC000DF93EC01FB018281882309F43CC1C4300F
:102AD000FDE5DF0760F4CB3F9CE5D90788F49E0154
:102AE00022503C452431310508F02EC109C0C236C0
:102AF000EDE5DE0729F0C63AFDE5DF0709F024C160
:102B00000E94840D90937C0280937B02C1318CE5FE
:102B1000D80709F4C6C008F042C0C930ECE5DE07AA
:102B200009F49BC000F5C5308CE5D80709F485C0D1
:102B300078F4C330ECE5DE0709F478C008F07AC019
:102B4000C230DC4509F0F5C080917B028160EFC0A6
:102B5000C7309CE5D90709F478C008F07AC08091A5
:102B60007B028061E4C0CD30FCE5DF0709F487C05B
:102B700058F4CB309CE5D90709F479C008F07BC044
:102B800080917B0288606FC0CF30FCE5DF0709F4DD
:102B900080C008F082C080917B02877FC8C0CE3F92
:102BA0009CE5D90709F471C000F5C531FCE5DF07E4
:102BB00009F485C068F4C3319CE5D90709F475C0F0
:102BC00008F095C00E94350780917B028F77AFC0D7
:102BD000CC3FFCE5DF07A9F108F054C0CB3FDC4552
:102BE00009F0A7C080917C0240C0C230EDE5DE074D
:102BF00009F489C058F4C1158DE5D80709F45AC005
:102C000008F069C080917C0282602FC0C236EDE579
:102C1000DE0709F47CC0C63AFDE5DF0709F481C090
:102C2000C330DD4509F085C080E06EC080917B0235
:102C300082607DC080917B0216C080917B0288609B
:102C400076C080917C0282604FC080917B0280625E
:102C50006EC080917B0280646AC00E9435078091BB
:102C60007B02806864C0846062C081603DC08091E6
:102C70007B028E7F5CC080917B028D7F58C08091EB
:102C80007B0216C080917C0218C080917C028D7FEF
:102C90002BC080917B028F7E4AC080917B028F7D0A
:102CA00046C080917B028F7B42C080917B02877FF0
:102CB0008B7F3DC080917C028D7F8E7F15C080917F
:102CC0007B0282FB222720F991E0922790FB82F978
:102CD00090FB83F92CC080917C02982F9095917085
:102CE0008E7F892B90FB81F980937C0222C00E9409
:102CF000350780917B0287FB222720F991E09227FC
:102D000090FB87F914C081E00E941B0E12C08091D5
:102D10007B0284FB222720F991E0922790FB84F923
:102D200006C080917B02982F909590FB80F980934C
:102D30007B0280917B0290917C020E94950D0E9403
:102D4000350780E001C081E0DF91CF9108958FE8E1
:102D500091E00197F1F700C0000008950C9415026E
:102D600023982B9A22982A9A0E94A71683B183FB54
:102D7000882780F91A9902C090E001C092E0892B5F
:102D8000809361020895E0916102EE0FEE0FE093EF
:102D9000610243B143FB882780F990E043B142FBD5
:102DA000222720F930E042FF02C022E030E0822BEF
:102DB000932B8E2B809361028F70E82FF0E0EF56FB
:102DC000FE4F908180916002890F809360021816F7
:102DD0005CF480915F028F5F80935F0260E080E02F
:102DE0000E94AE1681E001C080E09091600297FFE2
:102DF0000AC080915F02815080935F0261E080E0B1
:102E00000E94AE1681E0109260020895CF93DF9386
:102E100086319C4541F5EB010E94880C982F8A81F0
:102E20002091020130910301882379F09A7A81E0A0
:102E300009F480E080936202911102C069E201C04E
:102E400065E3C9010E9499180AC08091620281114C
:102E500002C069E201C065E3C9010E949B180E949B
:102E6000CA0C80E001C081E0DF91CF9108950F93FB
:102E70001F93CF93DF93C42FD22FFC01828188232D
:102E8000C9F0409365020E944019909364028093B8
:102E9000630280E28C0F883008F057C0C77081E071
:102EA00001C0880FCA95EAF7DF91CF911F910F916A
:102EB0000C94920480916502481330C080916302A3
:102EC000909164020E945819883C910538F510E2EF
:102ED0001D0FCD17B9F080E28C0F883040F4C77019
:102EE00081E001C0880FCA95EAF70E949904183062
:102EF00028F581E09D2F977001C0880F9A95EAF719
:102F00000E949204802F0E9489041830F0F4D77038
:102F100081E001C0880FDA95EAF70AC080E28C0FE1
:102F2000883098F4C77081E001C0880FCA95EAF72D
:102F3000DF91CF911F910F910C949904802FDF9115
:102F4000CF911F910F910C948904DF91CF911F9124
:102F50000F9108950F939C01CB01243F4CE534075A
:102F600031F188F4293DFCE53F07D9F02A3D4CE5D5
:102F7000340779F1283D3C45A9F506E221EE41EE02
:102F800068ED7CE52BC0263FFCE53F07E1F0A8F0AB
:102F9000273F3C4539F507E225EE46EE67EF7CE535
:102FA0001DC007E225EE45EE69ED7CE517C006E29F
:102FB00021EE40EE64EF7CE511C007E225EE44EE21
:102FC00065EF7CE50BC006E221EE42EE66EF7CE5A4
:102FD00005C008E221E045EE6AED7CE50E94371766
:102FE00080E008C0FC018281882319F010926502FC
:102FF00001C081E00F9108959093A3018093A201F5
:10300000089590936B0280936A020895E0916A029A
:10301000F0916B02309721F00190F081E02D09943E
:1030200080E00895E0916A02F0916B02309721F000
:103030000280F381E02D09940895E0916A02F091F5
:103040006B02309739F022E0DC012C930480F5818B
:10305000E02D0994089520916802309169022817A3
:10306000390771F09093690280936802E0916A02D7
:10307000F0916B02309721F00680F781E02D0994E2
:10308000089520916602309167022817390771F080
:103090009093670280936602E0916A02F0916B025E
:1030A000309721F00084F185E02D09940895FC010A
:1030B000329697E080E0915029F021912223D9F3B4
:1030C0008F5FF9CF0895662349F0FC013296089688
:1030D0002191621729F0E817F907D1F780E00895E8
:1030E00081E008959C01FC0132969FEF80E04191C0
:1030F000461789F09F3F19F4411101C0982F8F5F47
:103100008630A9F79F3F39F0F901E90FF11D97FDCE
:10311000FA956283089508959C012A5F3F4FFC0150
:103120004281461301C01282019682179307B9F7B4
:1031300008950C9472180C948C18029626E0FC01E9
:1031400011922A95E9F7089508950C94A41883E044
:1031500080936C020C94A518811102C081E001C01B
:1031600082E080936C020C94A5180C94AC1881E05A
:1031700080936C020C94A5180C94B71808950C94C5
:10318000BE180C94BF180C94BE180C94BE180C9466
:10319000BE18CF930E94C5180E9437120E94C31810
:1031A000C0E08C2F0E946111892B29F4CF5FC630BB
:1031B000C1F780E001C081E0CF91089508951F928A
:1031C0000F920FB60F9211248F939F93AF93BF93DB
:1031D00080916D02811113C08091950290919602A9
:1031E000A0919702B09198024196A11DB11D8093C4
:1031F000950290939602A0939702B0939802BF9184
:10320000AF919F918F910F900FBE0F901F901895C7
:1032100080919D02843031F10E94D80210926D029B
:1032200020E488E190E00FB6F894A89580936000C0
:103230000FBE2093600083B7817F846083BF83B714
:10324000816083BF7894889583B78E7F83BF0FB6E4
:10325000F894A89580916000886180936000109236
:1032600060000FBE08950E9435070C94DC0282E0D6
:1032700084BD93E095BD9AEF97BD80936E0008954D
:103280002FB7F8948091950290919602A0919702A1
:10329000B09198022FBF08952FB7F89460919502CE
:1032A0007091960280919702909198022FBF089595
:1032B0009C014FB7F8948091950290919602A0914D
:1032C0009702B09198024FBF821B930B0895789498
:1032D0001F920F920FB60F9211248F939F93AF936B
:1032E000BF938091950290919602A0919702B09120
:1032F00098020196A11DB11D8093950290939602AC
:10330000A0939702B0939802BF91AF919F918F9134
:103310000F900FBE0F901F90189581E08093E000F2
:1033200080E28093D8001092C9008FE19EE401975B
:10333000F1F700C0000087E090EBDC018093A6026B
:103340009093A702A093A802B093A9029CE088E101
:103350000FB6F894A895809360000FBE909360001C
:10336000FFCF809179020895089522E02093E9002B
:103370002FEF3091E800215035FD06C035ED3A952C
:10338000F1F700002111F5CF2091E80025FF0BC0D7
:1033900040E050E066E070E00E94DF1B8091E800B2
:1033A0008E778093E8000895CF93DF9321E02093F8
:1033B000E9002FEF3091E800215035FD06C035EDD2
:1033C0003A95F1F700002111F5CF2091E80025FF93
:1033D00014C0EC0140E050E068E070E00E94DF1BA8
:1033E0008091E8008E778093E80088E0FE01A1E7F5
:1033F000B2E001900D928A95E1F7DF91CF910895A7
:1034000080936E027093700260936F0280919D02B0
:10341000843001F582E08093E9008FEF9091E8001D
:10342000815095FD06C095ED9A95F1F70000811148
:10343000F5CF8091E80085FF0DC040E050E063E0EB
:1034400070E08EE692E00E94DF1B8091E8008E77AC
:103450008093E8000895BC0184E00C94001ABC013C
:1034600083E00C94001A80919C02811109C00E9493
:10347000701D0E94CD1D8091E20084608093E20067
:10348000089510929C0208950C94BC1860919902C2
:1034900081E0611101C080E00C94A71890919D0219
:1034A00081E0943009F080E0609199020C94AC18AE
:1034B00042E061EC81E00E94E91C42E261EC82E0C2
:1034C0000E94E91C90919D0281E0943009F080E017
:1034D000609199020C94B51880919F02833009F491
:1034E00061C030F4813071F0823009F49AC00895DF
:1034F0008A3009F486C08B3009F46CC0893009F039
:10350000A8C020C080919E02813A09F0A2C080919B
:10351000E800877F8093E8008091A2029091A30247
:10352000892B21F468E081E792E003C060E080E04D
:1035300090E070E00E942A1C8091E8008B778093D5
:10354000E800089580919E02813209F082C0809146
:10355000A2029091A302029708F07BC08091E8003C
:10356000877F8093E8008091E80082FD05C080910C
:103570009D028111F8CF6DC02091F3008091F2007F
:1035800090E0922B029731F48091F100813011F09C
:10359000863021F48091F100809379028091E800D7
:1035A0008B7753C080919E02813A09F052C080917E
:1035B000A2029091A302892B09F04BC08091E800F0
:1035C000877F8093E8008091E80080FFFCCF8091A6
:1035D000180136C080919E028132D9F58091A202F5
:1035E0009091A302892BA9F58091E800877F8093B1
:1035F000E8000E941E1D8091A002809318010C9487
:10360000350780919E02813221F58091E800877F05
:103610008093E8000E941E1D8091A10280937A028F
:10362000089580919E02813AA1F48091E800877FFD
:103630008093E8008091E80080FFFCCF80917A02BF
:103640008093F1008091E8008E778093E8000C94DD
:103650001E1D089584B7877F84BF0FB6F894A89580
:1036600080916000886180936000109260000FBEBE
:1036700090E080E80FB6F894809361009093610029
:103680000FBE0C94B7180E94701D0E94CD1DE2EE73
:10369000F0E080818460808378940C9462208CE0D8
:1036A00091E00C94011880919D028530A9F48091DD
:1036B0009D02853079F40E94081980919B0288232D
:1036C000B1F30E94C918882391F30E94C91B0E947C
:1036D0003507EDCF0C943319089508950C94701BA1
:1036E000292F332723303105C9F060F4213031050B
:1036F00081F02230310509F044C08BE390E02EEADE
:1037000032E043C021323105E1F02232310549F186
:1037100038C082E190E029EE32E037C0992781304D
:10372000910549F028F0029761F5E8E5F2E005C05F
:10373000EAEAF2E002C0E6E9F2E0849190E09F015B
:1037400024C06115710541F061307105D1F489E043
:1037500090E029ED32E019C089E090E020EC32E001
:1037600014C06115710541F06130710551F48BE7AA
:1037700090E02BEF32E009C080E490E026E733E0F0
:1037800004C080E090E020E030E0FA013183208343
:10379000089580E189BD82E189BD09B400FEFDCFB5
:1037A0008091D8008F7D8093D8008091E000826066
:1037B0008093E0008091E00081FDFCCF0895CF92DE
:1037C000DF92EF92FF920F931F93CF93DF93EC0161
:1037D0008B017A010E943D1D811133C0E114F10477
:1037E00039F0F70180819181081B190BC80FD91F8F
:1037F000C12CD12C0115110519F18091E80085FD2E
:1038000016C08091E8008E778093E800E114F104FF
:1038100049F0F70180819181C80ED91ED182C08202
:1038200085E00FC00E943D1D882321F30AC08991C5
:103830008093F10001501109FFEFCF1ADF0ADACFB0
:1038400080E0DF91CF911F910F91FF90EF90DF907B
:10385000CF9008952091A4023091A5022617370732
:1038600048F06115710539F42091E8002E77209316
:10387000E80001C0B901FC0120E06115710579F192
:1038800080919D028823F1F18530F1F18091E8006B
:1038900083FD3CC08091E80082FD2EC08091E8004D
:1038A00080FFEBCF2091F3008091F20090E0922B0B
:1038B0006115710551F08830910538F421912093FC
:1038C000F100615071090196F3CF21E0089709F0EA
:1038D00020E08091E8008E778093E800CECF211120
:1038E000CFCF0AC080919D02882361F0853061F0BE
:1038F0008091E80083FD0AC08091E80082FFF2CF4A
:1039000080E0089582E0089583E0089581E00895BD
:103910002091A4023091A5022617370748F06115BF
:10392000710539F42091E8002E772093E80001C05A
:10393000B901FC0120E06115710591F180919D02B2
:10394000882309F440C0853009F43FC08091E80025
:1039500083FD3DC08091E80082FD2FC08091E8008A
:1039600080FFE9CF2091F3008091F20090E0922B4C
:103970006115710559F08830910540F42491209328
:10398000F1003196615071090196F2CF21E008975C
:1039900009F020E08091E8008E778093E800CBCF9B
:1039A0002111CCCF0AC080919D02882361F085301F
:1039B00061F08091E80083FD0AC08091E80082FFF9
:1039C000F2CF80E0089582E0089583E0089581E0D9
:1039D0000895982F973068F59093E900981739F07B
:1039E0007091EC002091ED005091F00003C0242F65
:1039F000762F50E021FD02C09F5FECCF3091EB00AD
:103A00003E7F3093EB003091ED003D7F3093ED0031
:103A10003091EB0031603093EB007093EC00209319
:103A2000ED005093F0002091EE0027FDE5CF80E0FF
:103A300008958F708093E90081E0089580919E023F
:103A400087FF11C08091E80082FD05C080919D0232
:103A50008111F8CF11C08091E8008B770BC0809165
:103A60009D02882349F08091E80080FFF8CF809183
:103A7000E8008E778093E80008952091E40030916B
:103A8000E50095E64091EC00842F817040FF23C053
:103A90008091E80080FD1DC080919D02882399F0EF
:103AA000853099F08091EB0085FD11C04091E400D4
:103AB0005091E5002417350729F3915011F09A0130
:103AC000E1CF84E0089582E0089583E0089581E0E5
:103AD000089580E008954091E80042FFDDCF089509
:103AE0000E94DE1D0E94E61DE0EEF0E08081816014
:103AF0008083E8EDF0E080818F77808319BCA7EDAB
:103B0000B0E08C918E7F8C9380818F7E8083109229
:103B10009C0208950F931F93CF93DF930E94DE1DA5
:103B20000E94E61DC8EDD0E088818F778883888168
:103B30008068888388818F7D888319BC10929D025C
:103B40001092990210929B0210929A0200EE10E0DD
:103B5000F80180818B7F808388818160888342E047
:103B600060E080E00E94E91CE1EEF0E080818E7F61
:103B70008083E2EEF0E080818160808380818860D4
:103B80008083F80180818E7F808388818061888333
:103B9000DF91CF911F910F910895E8EDF0E08081C2
:103BA0008F7E8083E7EDF0E080818160808384E018
:103BB00082BF81E080939C020C948A1DE8EDF0E0C6
:103BC00080818E7F80831092E20008951092DA0047
:103BD0001092E10008951F920F920FB60F921124D8
:103BE0002F933F934F935F936F937F938F939F9305
:103BF000AF93BF93EF93FF938091E10082FF0BC0DF
:103C00008091E20082FF07C08091E1008B7F80936A
:103C1000E1000E9461208091DA0080FF1FC0809146
:103C2000D80080FF1BC08091DA008E7F8093DA007D
:103C30008091D90080FF0DC080E189BD82E189BDFE
:103C400009B400FEFDCF81E080939D020E94331AEB
:103C500005C019BC10929D020E94411A8091E1009A
:103C600080FF19C08091E20080FF15C08091E200C2
:103C70008E7F8093E2008091E20080618093E20079
:103C80008091D80080628093D80019BC85E0809331
:103C90009D020E94461A8091E10084FF30C080910D
:103CA000E20084FF2CC080E189BD82E189BD09B4B6
:103CB00000FEFDCF8091D8008F7D8093D800809149
:103CC000E1008F7E8093E1008091E2008F7E8093FF
:103CD000E2008091E20081608093E200809199028D
:103CE000882311F084E007C08091E30087FD02C0C3
:103CF00081E001C083E080939D020E944E1A809172
:103D0000E10083FF29C08091E20083FF25C08091FC
:103D1000E100877F8093E10082E080939D02109212
:103D200099028091E1008E7F8093E1008091E20012
:103D30008E7F8093E2008091E20080618093E200B8
:103D400042E060E080E00E94E91C8091F000886021
:103D50008093F0000E94441AFF91EF91BF91AF91C0
:103D60009F918F917F916F915F914F913F912F9193
:103D70000F900FBE0F901F9018951F920F920FB6C5
:103D80000F9211242F933F934F935F936F937F93E1
:103D90008F939F93AF93BF93CF93DF93EF93FF9353
:103DA000C091E900CF708091EC00D82FD17080FDD8
:103DB000D0E81092E9008091F000877F8093F000B6
:103DC00078940E94011F1092E9008091F0008860B1
:103DD0008093F000CD2BCF70C093E900FF91EF915D
:103DE000DF91CF91BF91AF919F918F917F916F9113
:103DF0005F914F913F912F910F900FBE0F901F90A9
:103E000018951F93CF93DF93CDB7DEB7AA970FB660
:103E1000F894DEBF0FBECDBFEEE9F2E08091F10075
:103E2000819322E0E63AF207C9F70E946C1A80916A
:103E3000E80083FF2EC180919E0290919F02492F3E
:103E400050E04A30510508F024C1FA01EE59FF4F05
:103E50000C949120803821F0823809F01AC108C0F2
:103E600080919A0290919B02992389F082600FC001
:103E70008091A2028F70873008F00BC18093E90017
:103E80008091EB0085FB882780F91092E9009091E2
:103E9000E800977F9093E8008093F1001092F10082
:103EA000D1C0282F2D7F09F0F4C0882319F082306B
:103EB00061F0EFC08091A002813009F0EAC0933038
:103EC00009F080E080939B022EC08091A0028111B6
:103ED0002AC08091A2028F702FEF280F263008F0A1
:103EE000D8C08093E9002091EB0020FF1CC09330E4
:103EF00021F48091EB00806214C09091EB009061FE
:103F00009093EB0021E030E0A90102C0440F551F5F
:103F10008A95E2F74093EA001092EA008091EB0064
:103F200088608093EB001092E9008091E800877F21
:103F30008093E8000E941E1DACC08111AAC01091A0
:103F4000A0021F778091E3008078812B8093E300AB
:103F50008091E800877F8093E8000E941E1D809179
:103F6000E80080FFFCCF8091E30080688093E3004D
:103F7000111102C082E001C083E080939D0289C0DC
:103F80008058823008F085C08091A0029091A102F3
:103F90008C3D53E0950779F583E08A838AE2898333
:103FA0004FB7F894DE01139620E03EE051E2E32F94
:103FB000F0E050935700E49120FF03C0E295EF70CA
:103FC0003F5FEF708E2F90E0EA3010F0C79601C08F
:103FD000C0968D939D932F5F243149F74FBF8091F9
:103FE000E800877F8093E8006AE270E0CE010196E6
:103FF0000E942A1C16C06091A2027091A302AE0119
:104000004F5F5F4F0E946E1BBC01892B09F441C0BA
:104010009091E800977F9093E80089819A810E94AF
:10402000881C8091E8008B778093E80032C080384C
:1040300081F58091E800877F8093E8008091990264
:104040008093F1008091E8008E7772CF811121C0BA
:104050008091A0029091A10299270297D4F48091B7
:10406000E800877F8093E8008091A0028093990206
:104070000E941E1D80919902811106C08091E3006B
:1040800087FD02C081E001C084E080939D020E9410
:10409000581A8091E80083FF0AC08091E800877F6A
:1040A0008093E8008091EB0080628093EB00AA96F9
:1040B0000FB6F894DEBF0FBECDBFDF91CF911F9139
:1040C00008950895CF9380919D028823A1F0C09117
:1040D000E900CF709091EC00892F817090FD80E80D
:1040E000C82B1092E9008091E80083FD0E94011F17
:1040F000CF70C093E900CF91089597FB072E16F477
:10410000009407D077FD09D00E94972007FC05D0C6
:104110003EF4909581959F4F0895709561957F4FDE
:104120000895EE0FFF1F0590F491E02D0994AA1B4E
:10413000BB1B51E107C0AA1FBB1FA617B70710F092
:10414000A61BB70B881F991F5A95A9F780959095C4
:10415000BC01CD010895FB01DC0104C08D910190EB
:10416000801921F441505040C8F7881B990B0895DD
:10417000F999FECF92BD81BDF89A992780B508952F
:10418000A8E1B0E042E050E00C94EC20262FF99931
:10419000FECF92BD81BDF89A019700B4021639F0A6
:1041A0001FBA20BD0FB6F894FA9AF99A0FBE089577
:1041B0000396272F0E94C7200E94C620252F0E9409
:1041C000C720242F0C94C7200196272F0E94C720B8
:1041D0000C94C620DC01CB01FC01F999FECF06C08E
:1041E000F2BDE1BDF89A319600B40D9241505040B5
:0841F000B8F70895F894FFCF21
:1041F800C8002C02280850011E0A1401B119D4194C
:10420800B5192F1A2B1AB41901E200E900EA00B512
:1042180000B600B700CD008301CC008A019201945A
:10422800012102230224022502260227022A02B3C0
:1042380000B4006F007000818283E200E900EA00A8
:10424800B500B600B700CD008301CC008A01920109
:1042580094012102230224022502260227022A02AF
:10426800B300B4006F0070008182839594969734F0
:1042780035366667F7F6F5F4F1F0C6379091929304
:104288003000FF0100010000FFFF0000010001FFF6
:02429800000024
:00000001FF
